:100000004FC000005DC000005BC0000059C0000090
:1000100057C0000055C0000053C0000051C0000090
:100020004FC000004DC000004BC0000049C00000A0
:1000300047C0000045C0000043C0000041C00000B0
:100040003FC000003DC000003BC0000039C00000C0
:1000500037C0000035C0000033C0000031C00000D0
:100060002FC000002EC000002BC0000029C00000DF
:1000700027C0000025C0000023C0000021C00000F0
:100080001FC000001DC000001BC0000019C0000000
:1000900017C0000015C0000013C0000011C0000010
:1000A00011241FBECFEFCDBFDFE3DEBF2CE3A0E006
:1000B000BCE301C01D92A430B207E1F72AD09BC077
:1000C0009FCF1F920F920FB60F9211248F939F9381
:1000D000AF93BF938091003C9091013CA091023C72
:1000E000B091033C0196A11DB11D8093003C9093FB
:1000F000013CA093023CB093033C81E08093A60AAC
:10010000BF91AF919F918F910F900FBE0F901F9055
:10011000189588ED90E084BF90936100809102066D
:1001200086608093020680910006816080930006BD
:10013000809102068F7C8065809302061092E20512
:1001400082E08093E40581E08093030A8EEF809340
:10015000270A8093260A80E880932D0A80932B0A31
:100160008093290A80932C0A80932A0A8093280A74
:100170008BE08093000A87E08093E505E0E8FAE0F1
:1001800037E02EEF90E885E03183248795878083E0
:100190007096E03C4AE0F407B9F71092A10A8FE7A5
:1001A0009EE38093AC0A9093AD0A8091A50A81608A
:1001B0008093A50A1092A00A8091A00A8160809382
:1001C000A00A789482E08093010412E0C0E0D0E0BD
:1001D0008091000481FF06C0109305042097C1F3AD
:1001E0000FDFF6CF9FB7F894809111048860809359
:0A01F00011049FBFF3CFF894FFCF76
:00000001FF
